:020000040000FA
:08000000803102288731FC2F3A
:100C4400863137268631262E20008C1C2A2E2B2E08
:100C54002F2E86314E268631262E87312527863142
:100C6400262E262E262E803102286A302100990055
:100C74001D14013023008C00033021008C0022005D
:100C84008C0120008C0123008D0121008D012200A4
:100C94008D0120008D010800F00121009E131D1319
:100CA4009D121D129D111D110D30F100FC30890B98
:100CB400592EF10B592E21009D141C08F1007108C6
:100CC400F0007008031D672E682E722E20000D1090
:100CD4008D100D118D110D128D120D138D13242FE6
:100CE40002307002031C772E782E882E203070027A
:100CF40003187D2E7E2E882E20000D148D100D11CC
:100D04008D110D128D120D138D13242F21307002AD
:100D1400031C8D2E8E2E9E2E403070020318932EAF
:100D2400942E9E2E20000D108D140D118D110D1278
:100D34008D120D138D13242F40307002031CA32E2B
:100D4400A42EB42E603070020318A92EAA2EB42E3D
:100D540020000D108D100D158D110D128D120D1317
:100D64008D13242F60307002031CB92EBA2ECA2EA4
:100D7400803070020318BF2EC02ECA2E20000D1022
:100D84008D100D118D150D128D120D138D13242F31
:100D940080307002031CCF2ED02EE02EA0307002C3
:100DA4000318D52ED62EE02E20000D108D100D1117
:100DB4008D110D168D120D138D13242FA03070027A
:100DC400031CE52EE62EF62EC03070020318EB2E1F
:100DD400EC2EF62E20000D108D100D118D110D121C
:100DE4008D160D138D13242FC0307002031CFB2E9F
:100DF400FC2E0C2FE03070020318012F022F0C2F51
:100E040020000D108D100D118D110D128D120D1766
:100E14008D13242FE0307002031C112F122F242F66
:100E240020000D108D100D118D110D128D120D134A
:100E34008D17242F242F242F242F242F242F242FC5
:100E4400242F242F0800F00121009E131D139D124E
:100E54001D129D111D110D30F100FC30890B302F36
:100E6400F10B302F21009D141C08F1007108F000D3
:100E74007008031D3E2F3F2F492F20000D108D10A9
:100E84000D118D110D128D120D138D13FB2F0230C8
:100E94007002031C4E2F4F2F5F2F20307002031857
:100EA400542F552F5F2F20000D148D100D118D110F
:100EB4000D128D120D138D13FB2F21307002031CA4
:100EC400642F652F752F4030700203186A2F6B2F23
:100ED400752F20000D148D140D118D110D128D120E
:100EE4000D138D13FB2F40307002031C7A2F7B2FC0
:100EF4008B2F603070020318802F812F8B2F2000DE
:100F04000D148D140D158D110D128D120D138D13DD
:100F1400FB2F60307002031C902F912FA12F803083
:100F240070020318962F972FA12F20000D148D14F3
:100F34000D158D150D128D120D138D13FB2F803091
:100F44007002031CA62FA72FB72FA030700203181E
:100F5400AC2FAD2FB72F20000D148D140D158D154A
:100F64000D168D120D138D13FB2FA0307002031C70
:100F7400BC2FBD2FCD2FC03070020318C22FC32F3A
:100F8400CD2F20000D148D140D158D150D168D16F5
:100F94000D138D13FB2FC0307002031CD22FD32FDF
:100FA400E32FE03070020318D82FD92FE32F20004D
:100FB4000D148D140D158D150D168D160D178D131D
:100FC400FB2FE0307002031CE82FE92FFB2F2000D9
:100FD4000D148D140D158D150D168D160D178D17F9
:100FE400FB2FFB2FFB2FFB2FFB2FFB2FFB2FFB2FAD
:0C0FF400FB2F0800F00120008631222EA7
:020000040001F9
:04000E00A4C9FFDCA6
:00000001FF
